:020000040000FA
:100000008028820700340034003401340034003486
:1000100000340A34003400340034643400340034D2
:100020000334E8340034003427341034003401340D
:100030008634A03400340F344234403400349834D1
:1000400096348034820707341234033436340B3448
:10005000183403343A3403341C3400343E340D3441
:1000600021340334423482070A3409340834063414
:100070000534043402340134820753347734653450
:1000800065347034473465346E340034203456346B
:100090006534723431342E343134203400345334E6
:1000A0007434613472347434003445346E346434DE
:1000B0000034533474346534703400344D34613456
:1000C00072346B34653472340034533477346534AD
:1000D0006534703469346E346734003442346134CA
:1000E0006434203445346E346434003420344B346A
:1000F00048347A340034433441344C3420340034AE
:100100008B0107309F009801831698018C019F0195
:100110008113FB30850086018312AD01AE01AF0172
:10012000B001B101932293220515AE220E30DE00FC
:10013000CE222930840000309F23D101D50105084B
:10014000D00003305005CF00501E2F227C230030FA
:10015000BC200430BC20DA20031CB3283F233130FC
:10016000D422D023A9280830BC200C30BC208E23F8
:10017000E6207C231E22A728DA002220DE00C923E5
:100180003F235A08013E2220D422D0235A08023E9F
:100190002220D800030116223F235A08033E2220C2
:1001A000DD0019239222A421551AD8283621D328FC
:1001B000551208003608AD003708AE003808AF0009
:1001C0003908B0003D30840011210800D5143E30BC
:1001D000DD005522323029213A300C2142300C21E9
:1001E0003F232830D42205113630DD0055222D3032
:1001F000DD00EF21551A0929932245308400112191
:10020000031805153F213D30840011210318F32800
:10021000F928D50105150800DD0055225D082921C2
:10022000080000083002031C2829031D2829840324
:1002300000082F02031C2829031D28298403000815
:100240002E02031C2829031D2829840300082D02DF
:10025000080084002D088000840A2E088000840A8B
:100260002F088000840A300880000800D1183A293D
:1002700088213C293F215E21192392220800D701C1
:100280005D088400320880070330D30058218403BE
:100290008403330880070230D300582184033408D4
:1002A0008007840A031C5529800A35088007080046
:1002B000570D840A8007D30B5829080003305D07C7
:1002C000840003300002031C8729031D7A2984035C
:1002D00093300002031C8729031D7A298403873089
:1002E0000002031C8729031D7A29840300300002C1
:1002F000031C87295D08840000308000840A873051
:100300008000840A93308000840A03308000080053
:1003100098213F2103305D078400801F96298001CA
:1003200084038001840380018403800198210800F4
:10033000B209B309B409B509B20FA329B30FA329B0
:10034000B40FA329B50A0800D321551AD2290508EC
:10035000D000E52305085006031DA42903305005ED
:10036000CE004F060319A4290310CF0D4E08CF0667
:100370004F080239D2005106D101CF18C7294E08C3
:10038000CF00DC035C18A429DC18A429D029023092
:10039000D1004E08CF00DC0A5C18A429DC18A4297F
:1003A0004E08CF000800D518132A051AEF29851D1D
:1003B000FB292030D6005510DC23051AEB29851DBA
:1003C000FB29D603031DDC29013016220430D60098
:1003D0005514D511DC290130D519132A0E2A851997
:1003E000132ADC238519F929D518F129051EFB29C3
:1003F000F1295516132A2030D6005510D515DC23C7
:10040000051A0D2A85190D2AD603031DFF29FF3071
:1004100016220430D6005514FF29FF305518132A30
:100420001622051ED329D511551008005807073983
:10043000D8003320D9001E22192308000430D3002D
:10044000353084005808D7000310D70DD70D570852
:10045000012080008403D70AD30B272A0800D51473
:100460003630840004309F233630DD0019238C3071
:100470005A233E30D4229222A421051A4F2AB501D4
:10048000B401B3010430D01D8030B200D118492A24
:1004900098212930DD003F213630DD003B2A29300C
:1004A00084000301A923D5100800AD01AE01AF01FE
:1004B000B001B1012030D3002908A5002A08A60008
:1004C0002B08A7002C08A8005D0884000310251C39
:1004D000832A0008AE07031C722AAF0F722AB00FDE
:1004E000722AB10A840A0008AF07031C7A2AB00FE7
:1004F0007A2AB10A840A0008B007031C802AB10ACC
:10050000840A0008B107B10CB00CAF0CAE0CAD0CF6
:10051000A80CA70CA60CA50C5D08D30B652A01300E
:10052000B100080055222D3084000008C9000830B1
:10053000C800C90C031CA02A861506150611A32A9B
:10054000861106150611C80B992A840A3230040256
:10055000031C952A86178613C9230800D923033064
:1005600086000616D9230612033086000616DC2301
:100570000612033086000616DC23061202308600BF
:100580000616DF23061220305A2308305A23013082
:100590005A2306305A230E305A2308000030D42242
:1005A0000930D422CE230800DB003C20FF39031998
:1005B000DD2A5E23DB0A5B08D52A08002030C6004E
:1005C000A001A101A201A301A4015D08840000080B
:1005D000A500840A0008A600840A0008A700840A6F
:1005E0000008A8000310A50DA60DA70DA80D03185F
:1005F0002514A00DA10DA20DA30DA40DC603031D6E
:10060000022B0800203084000E23840A0E23840A63
:100610000E23840A0E23840A0E23F22A03300007D5
:10062000C700C719800030300007C700C71B800013
:100630000800DE2202305A2320305E23230E3723A7
:10064000230837232C305E23220E3723220837233A
:10065000210E37232E305E2321083723200E372327
:10066000200837233930D4223A23C92308000F3910
:10067000303E5E2B803059045A23C92308000130D4
:100680005A23080086018316083086008312061359
:100690008616FF30CC0006160608CB0006120000B6
:1006A0000000061600000612CC030319592BCB19C3
:1006B0004B2B0800CA00D4010613612BCA00541446
:1006C00006174223860183160030860083128612A5
:1006D000061354180617F03086054A0E0F398604A3
:1006E000061600000612F03086054A080F39860407
:1006F00006160000061208003630DD0084000830BF
:100700009F233A3084000C309F233E308400103009
:100710009F234230840014309F2308003630840029
:100720000830A9233A3084000C30A9233E308400DD
:100730001030A923423084001430A9230800F000AF
:100740000430D300C2238000F00A840AD30BA22B0A
:100750000800F0000430D3000008B323840AF00A34
:10076000D30BAC2B080083169A0070089B001C1555
:1007700055309D00AA309D009C149C18BD2B1C1167
:1007800083120800831670089B001C141A08831239
:100790000800F13086055E0886040800D323D323C1
:1007A000D323D3230800D623D6230800FF30CC0060
:1007B000E72B8030CC00E72B4030CC00E72B2030FB
:1007C000CC00E72B1030CC00E72B0230CC00FF3000
:0C07D000CD00CD0BE92BCC0BE72B080073
:084000005700330043004400A7
:02400E00213F50
:10420000DF006500DC0017008000960098000000C9
:10421000800084001E00000020000B002000000031
:104220006400000000000000D00047001F000000F4
:00000001FF
